:020000040800F2
:1000000058050020D900000875120008A711000843
:1000100000000000000000000000000000000000E0
:10002000000000000000000000000000BF120008F7
:100030000000000000000000BD120008C11200080E
:10004000EB000008EB000008EB000008EB000008E4
:10005000EB000008EB000008EB000008EB000008D4
:1000600000000000EB000008EB000008EB000008B7
:10007000EB000008EB00000800000000EB000008A7
:1000800000000000EB00000800000000000000007D
:10009000EB00000800000000EB000008EB00000887
:1000A000EB000008EB000008EB000008FD1800085A
:1000B0000D190008EB00000800000000000000001F
:1000C0000448854600F090F800480047E11A00080F
:1000D000C046C046580500200448804704480047F1
:1000E000FEE7FEE7FEE7FEE7FEE7FEE7391300085E
:1000F000C100000830B50B46014600202022012433
:1001000009E00D46D5409D4205D31D469540491B4B
:100110002546954040191546521E002DF1DC30BD94
:10012000F0B51FB40646002082B005464024019178
:1001300000901BE0019922460F46304600F042F83D
:10014000049A059B801A994110D3104619462246FD
:1001500000F028F8361A8F4101972246012000212D
:10016000009F00F01FF838184D4100902046641E93
:100170000028DFDC019B00982946324607B0F0BD1D
:10018000D2B201E00270401C491EFBD2704700222F
:10019000F6E710B513460A4604461946FFF7F0FF86
:1001A000204610BD10B5202A04DB0146203A9140BC
:1001B000002010BD914020239C1A0346E3401943C0
:1001C000904010BD10B5202A04DB0846203AD040EC
:1001D000002110BD0B46D340D0402024A21A9140EC
:1001E0000843194610BD0000064C0125064E05E0E7
:1001F000E36807CC2B430C3C98471034B442F7D348
:10020000FFF762FF481B0008681B0008704770B5C5
:100210000024014620314A79022A03D00421C16317
:10022000012418E0026813680E25AB4313600268CE
:1002300013685B085B001360436C1C2213400122AF
:1002400015469D40036C5D604A7100220A71816B06
:10025000002900D08847204670BD70B5044600F0E4
:10026000C7F80546601C00D0641C00F0C1F8401BB4
:10027000A042FAD370BD0000F8B500230124A2E02B
:1002800027469F403A4070D04D68022D01D0122D74
:1002900014D1DD08AD002D1800952D6A5E07AC461F
:1002A000F50E0F26AE46AE406546B543AC460E6928
:1002B0007546AE4065462E43009D2E624D68012D69
:1002C00005D0022D03D0112D01D0122D16D1856835
:1002D0000326AC465D00AE46AE406546B543AC462F
:1002E000CE687546AE4065462E43866046680D79F9
:1002F000BE43ED06ED0F9D403543456006685F0047
:100300000325BD40AE46AE430D79B446AE07B60FE9
:10031000BE4065462E430660C6687546AE438D688E
:10032000BD403543C5604D68ED004BD5294D6E6B22
:1003300026436E639E08284DB6007519AC46AD681D
:100340009E07360F0F27B740BD4305273F07B8422A
:1003500001D1002715E0214FB84201D1012710E05B
:100360001F4FB84202D102270BE02BE01D4FB842CD
:1003700001D1032705E01C4FB84201D1052700E059
:100380000627B7402F436546AF60184D2E684F686B
:100390009643FF0300D516432E606E684F68964360
:1003A000BF0300D516436E60AE684F689643FF02E8
:1003B00000D51643AE60EE684F689643BF0200D585
:1003C0001643EE605B1C0A681546DD4000D057E717
:1003D000F8BD000000100240000001400004005081
:1003E00000080050000C0050001C005000040140A8
:1003F00001480068704700001000002002480168B2
:10040000491C0160704700001000002010B508482A
:1004100000240168402211430160204600F00AF8E0
:10042000002801D0012401E000F01CF8204610BD96
:100430000020024070B5054609487D210024C9000E
:100440000068FFF757FE00F0F9FB002801D00124F7
:1004500004E000222946501E00F01AF8204670BD24
:10046000140000200448416B012211434163816B59
:10047000020411438163704700100240C106C90E97
:1004800001208840014908607047000000E100E059
:1004900010B500F0F1FE10BDF8B504460078544DDB
:1004A000800672D5524E0027403EB06BC00004D487
:1004B000B06BA9050843B06301274E480168C90520
:1004C00011D40168821511430160FFF791FF00907C
:1004D00005E0FFF78DFF0099401A642837D845489A
:1004E0000068C005F5D532680321090560680A4037
:1004F0000140914208D08103890F032904D131685A
:10050000890301D50120F8BD2A69032109040A40A5
:1005100022D0084090421FD0207880061CD5286940
:100520002A6988430121C9040A432A612A698A4346
:100530002A612861C0050FD5FFF75AFF009008E037
:10054000FFF756FF0099411A2B48814201D9032039
:10055000F8BD28698005F3D561688803800F0328FA
:1005600005D132680005824301400A4332602869A0
:10057000032261681204114008432861002F04D04F
:10058000B16B012000078143B1632078C00705D01B
:10059000E868A168800880000843E8602078800748
:1005A00005D5E8680C218843E1680843E8602078B5
:1005B000400706D5E868032189028843216908437A
:1005C000E8602078000706D5E8680321090388431E
:1005D00061690843E8602078000606D5E8680321D1
:1005E00089048843A1690843E8600020F8BD000041
:1005F000401002400070004088130000F8B50E461D
:1006000005007DD053480068C007C00FB0420AD231
:100610005048016849084900314301600068C0073B
:10062000C00FB04271D128784B4C800705D5E068E7
:10063000F0218843A9680843E0602878C00752D0B9
:100640006868022817D0032818D02168012818D01C
:100650008905002959DAE168890889000143E160C8
:10066000FFF7C6FE69680746022912D003291CD08D
:10067000012926D033E021688903EAE7216889014E
:10068000E7E74907E5E7FFF7B3FEC11B33488142BF
:1006900023D8E0680007800F0228F4D123E0FFF799
:1006A000A7FEC11B2D48814217D8E0680007800FC4
:1006B0000328F4D117E0FFF79BFEC11B27488142B6
:1006C0000BD8E0680007800F0128F4D10BE0FFF79A
:1006D0008FFEC11B2148814201D90320F8BDE0688B
:1006E0000007800FF3D11B480168C907C90FB14249
:1006F0000DD901684908490031430160006800E0F4
:1007000003E0C007C00FB04201D00120F8BD287837
:10071000400706D5E068072109028843E9680843D5
:10072000E0602878000707D5E0680721C902884300
:100730002969C9000843E06000F036F8E168084A1A
:100740000906090F515CC840064908600020FFF700
:1007500071FEF8BD00200240001002408813000026
:10076000241B000814000020044805490068C968DB
:10077000044A4905490F515CC840704714000020E5
:10078000001002403D1B0008044805490068C96884
:10079000044A8904490F515CC84070471400002086
:1007A000001002403D1B000810B5184AD1680C200B
:1007B000084004280BD0082810D00C2810D050680E
:1007C0000004410F0120C003491C884010BD10687F
:1007D000C00601D50E4810BD0E4810BD0E4810BD14
:1007E00088020E4B000F185C0902D368890F491C60
:1007F000DB0301D5084A05E01268D20601D5044A98
:1008000000E0044A5043FFF775FC10BD00100240A1
:1008100000093D000024F40000127A00341B000897
:10082000FEB505007ED0FE4CE7680C20E668074068
:100830000120000406402878C00747D0082F05D0C3
:100840000C2F0AD101200004864206D120688003C3
:100850003CD568680028E5D038E0012069680004CC
:10086000814203D121680143216011E00523012267
:100870001B0492049942216802D111432160F1E7DF
:1008800081432160216801400091206890432060ED
:10089000686800280DD0FFF7ABFD009005E0FFF77A
:1008A000A7FD0099401A64287AD820688003F6D5FD
:1008B0000CE0FFF79DFD009005E0FFF799FD009922
:1008C000401A6428F0D820688003F6D4287880077E
:1008D00055D50923E868042F0DD00C2F01D1002E27
:1008E00009D000283BD02168994301432160FFF7DC
:1008F0007FFD064627E02168490701D5002891D0F1
:1009000061681F22120291432A6912021143616039
:100910002168994301432160FFF746FFE16809061A
:100920000A0F00E079E1BF49895CC840BE49086010
:100930000020FFF77FFD002872D120E0FFF758FD6F
:10094000801B0228B0D820684007F7D560681F21B7
:100950000902884329690902084360600FE02068A2
:10096000400840002060FFF743FD064604E0FFF723
:100970003FFD801B022897D820684007F7D42878CD
:10098000C0065FD5002F0CD0A869002849D0206888
:10099000FF21013108432060FFF72AFD06462DE0C4
:1009A000C0E02068800502D5A8690028A7D060684B
:1009B000072149038843296A084360606068297FEA
:1009C0000002000A090608436060286A410B012002
:1009D000C003491C8840E16809060A0F9149895CF7
:1009E000C840914908600020FFF724FD002817D176
:1009F00028E0FFF7FDFC801B0228A3D820688005B3
:100A0000F7D56068072149038843296A0843606075
:100A10006068297F0002000A09060843606011E04F
:100A2000E1E02168FF20013081432160FFF7E0FC15
:100A3000064604E0FFF7DCFC801B022872D8206821
:100A40008005F7D42878794E000724D568690028F6
:100A5000306910D0012108433061FFF7C9FC0090D4
:100A600005E0FFF7C5FC0099401A02285AD8306902
:100A70008007F6D50FE0400840003061FFF7B8FC72
:100A8000009005E0FFF7B4FC0099401A022849D80D
:100A900030698007F6D42878400765D50020029099
:100AA000A06BC00006D4A06B012109070843A06316
:100AB000012002905E480168C90511D401688215C1
:100AC00011430160FFF794FC009005E0FFF790FCF4
:100AD0000099401A642825D855480068C005F5D506
:100AE000FF20AA680130824203D13169014331619C
:100AF00011E001218902002A07D005231B029A4236
:100B000003D132690A433261EFE7326982433261CD
:100B1000306988433061A86800280FD0FFF768FC6F
:100B2000009007E05EE0FFF763FC0099411A41483E
:100B3000814257D830698005F5D50DE0FFF758FCA4
:100B4000009006E0FFF754FC0099411A39488142B1
:100B500048D830698005F5D40298002804D0A06BED
:100B6000012109078843A063686A002864D00C2F1C
:100B70003ED0012636060228206805D0B04320600A
:100B8000FFF736FC05462FE0B0432060FFF730FC4E
:100B9000074604E0FFF72CFCC01B022822D820687F
:100BA0008001F7D4E96AA86AE2680843296BFD234B
:100BB0001B049A4311430843E060206830432060DF
:100BC000FFF716FC054604E0FFF712FC401B022865
:100BD00008D820688001F7D52EE0FFF709FC401BFC
:100BE000022801D90320FEBD20688001F5D423E04E
:100BF0000128F8D0E06801210904AA6A0140914265
:100C00000BD10F218904EA6A0140914205D10321E9
:100C100089050840296B88420ED00120FEBD0000E6
:100C200000100240241B0008140000204010024065
:100C300000700040881300000020EFE7094910B55C
:100C4000401E884201D9012010BD074C606103217C
:100C5000081F00F011FB0020A06107202061002088
:100C600010BD0000FFFFFF0000E000E0F0B502460D
:100C70002032137E012B15D00127177602235376DD
:100C800005686C68AB687026B4430E6849682643F3
:100C90008024A34319436E6000688160577600206A
:100CA0001076F0BD0220F0BD70B5040005D02546D9
:100CB0002035687E002802D006E0012070BD0020AB
:100CC0002876204600F00AF802206876211D206868
:100CD00000F05CFB01206876002070BD00680449CC
:100CE000884204D10348816B10221143816370470D
:100CF000001000400010024070477047F8B50268CD
:100D00000446D0691168936805072D0F5BD0DD0795
:100D1000ED0FFF2621360E402E4367D0C60706D0C2
:100D2000CE0504D501261662E26F3243E2678707DB
:100D300002220426002F06DADF0704D027683A6271
:100D4000E76F3743E767470706D5DB0704D023681B
:100D50001E62E36F1343E367020709D520220A40AE
:100D60002A4305D0236808221A62E36F1343E3671E
:100D7000E26F002A2FD0800606D5880604D5216EA2
:100D8000002901D020468847E06F2168896849061C
:100D900001D4000724D5204600F0C4FB20688168F8
:100DA000490619D58168402291438160E06E002890
:100DB00012D020498163E06EFFF729FA00280AD09B
:100DC000E06E816B06E0850610D58D060ED5216E8E
:100DD0001CE020468847F8BD2046FFF78EFFF8BD8F
:100DE0002046FFF78AFF0020E067F8BDC50208D55E
:100DF0005B0206D50120000510622046FFF77CFF4C
:100E0000F8BD030605D50B0603D5616E0029E0D1B8
:100E1000F8BD4006FCD54806FAD5136820464021A7
:100E20008B431360202161670021616600F0BAF9ED
:100E3000F8BD00001115000810B5040003D0606F64
:100E4000002802D007E0012010BD002170200155CC
:100E5000204600F027F824206067206801684908D0
:100E600049000160204600F0C5FB0128ECD0606A13
:100E7000002802D0204600F0B5FA20684168092217
:100E8000D20291434160206881682A2291438160A7
:100E900020680168012211430160204600F008FB30
:100EA00010BD0000F0B587B0044614216846FFF776
:100EB0006EF9244F266800212348012202230324CF
:100EC0000425BE421AD1466B97033E434663C66A69
:100ED0001643C662C06A02AE1040059060020090E0
:100EE000019332C6052069460007FFF7C5F90022C5
:100EF00011461B20FFF7CCFA1B201EE0134FBE4209
:100F00001DD1866B01277F043E438663C66A164364
:100F1000C662C06A02AEC007C00F05900C200090E8
:100F2000019332C6052069460007FFF7A5F90022A4
:100F300011461C20FFF7ACFA1C20FFF79FFA07B000
:100F4000F0BD0000003801400010024000440040A5
:100F5000F0B5836F202B54D100290AD0002A08D085
:100F60008568DC01A54206D10369002B03D1CB07BC
:100F700001D00120F0BD034660331E7C012E40D01D
:100F800001261E744165014640310A834A830022CE
:100F9000FF260266A54204D10569002D13D11A4D22
:100FA0000AE07F27002D09D001263607B5420CD173
:100FB0000569002D05D03F258D8307E00569002DCB
:100FC00001D08F8302E08E8300E08A83C2672221F2
:100FD000816701688D68012635438D608168A14273
:100FE00002D1016900290AD0084901661A74006813
:100FF0000168FF222132114301600020F0BD044945
:10100000F3E70220F0BD0000FF0100009D1500087D
:101010004515000810B500680A49884211D10A48F0
:10102000017855290DD14178AA290AD141798079D1
:101030000902081881B204480838018003A000F0B2
:101040006DFC10BD0044004008000020646973740A
:10105000616E63653A25640A00000000FFB504462E
:10106000406F83B017460D4620285CD1002D0AD072
:10107000002F08D0A168C001814207D12069002853
:1010800004D1E80702D0012007B0F0BD204660304F
:101090000290007C012846D00298012101740020B2
:1010A000E06721206067FFF7A3F9264640360190EC
:1010B000378277820120A1680003814202D1206932
:1010C000002802D02F46002511E000270FE0002263
:1010D0008021204600F0E0FB002815D1002F15D01C
:1010E0002168387888627F1C708A401E7082708AFE
:1010F000019B002806980090E9D10022402120465B
:1011000000F0CAFB002808D00320BDE7288821682A
:10111000C005C00D8862AD1CE6E72020606702991B
:1011200000200874B0E70220AEE7000070B5436FFE
:10113000202B30D100290AD0002A08D08568DC0194
:10114000A54206D10369002B03D1CB0701D00120B2
:1011500070BD034660331E7C012E1CD001261E7418
:10116000C164014640310A824A8200214166C1675A
:1011700021224267A54202D10269002A09D0074A0A
:1011800042661974006801688022114301600020E2
:1011900070BD034AF4E7022070BD00005D1800082E
:1011A0001D1800087047FEE708B50448C16A01220F
:1011B0001143C162C06A1040009008BD0010024097
:1011C0001CB500240E4800940C49019401600721CD
:1011D0008460416001214461C160FFF765FD002822
:1011E00001D0FFF713F80094694605480194FFF712
:1011F0003DFD002801D0FFF709F81CBD001000409C
:101200001C00002010B50C480A490160E121490288
:10121000416000218160C16001618161C1610C2276
:10122000016242614162FFF707FE002801D0FEF72C
:10123000EDFF10BD003801405800002010B50C48EB
:101240000A4901604B210902416000218160C160AF
:1012500001618161C1610C22016242614162FFF75B
:10126000EBFD002801D0FEF7D1FF10BD0044004087
:10127000D8000020704700008307FF22DB0E9A4051
:101280008907090E994000280BDA0007000F08387B
:10129000830808489B001818C36993430B43C36134
:1012A0007047830804489B001B1818689043084344
:1012B0001860704700ED00E000E400E07047704700
:1012C00010B5FFF79BF810BD30B599B034216846D2
:1012D000FEF75DFF14210DA8FEF759FF1C2112A88F
:1012E000FEF755FF134801680322D2029143C2144E
:1012F0008918016002200090002410200994012523
:10130000049003956846FFF78BFA0F200D9080201C
:101310000F900E951094002111940DA8FFF76EF90F
:10132000032012901494159412A8FFF7B5F819B081
:1013300030BD000000700040104801688215114364
:101340000160C1680E4A1140C16001680D4A114038
:1013500001608168490849008160016801229204A6
:1013600091430160C168FD2212049143C1600021D4
:1013700001610549C0038860704700000010024009
:101380000C40FF88F6FFF6FE00ED00E070B5026845
:1013900001239B07114C124D984203D0A04201D06B
:1013A000A84203D17026B2434E683243984203D01C
:1013B000A04201D0A84204D103231B029A43CB6868
:1013C0001A4380239A430B691A4302608A68C262F7
:1013D000096881620121416170BD0000000801407F
:1013E0000014014010B5818CC90707D001684A6814
:1013F00001235B049A43836A1A434A60818C8907FC
:1014000007D501684A6801231B049A43C36A1A433B
:101410004A60818C490707D501684A6801239B040B
:101420009A43036B1A434A60818C090707D5016808
:101430004A680123DB039A43436B1A434A60818C59
:10144000C90607D50268916801231B039943836B82
:1014500019439160818C890607D501688A68012348
:101460005B039A43C36B1A438A60818C490612D589
:1014700003685A6801210905046C8A4322435A60B3
:10148000026C8A4207D10268516803235B059943C5
:10149000436C19435160818C090607D501684A687D
:1014A0000123DB04806C9A4302434A6010BD0000B4
:1014B000F8B500260446C667FEF79AFF0546206881
:1014C0000068124F000709D501212B46002249056B
:1014D0002046009700F0E0F900280DD12068006850
:1014E00040070BD501212B46002289052046009795
:1014F00000F0D2F9002801D00320F8BD2020606759
:10150000A067603426740020F8BD0000FFFFFF01D3
:1015100010B5806A0022014640314A834A82FFF7B3
:10152000ECFB10BD01680A68FF2321339A430A606F
:1015300001688A68520852008A6020218167002170
:101540000166704710B5014640318B8B846F02688D
:10155000222C04D0906908210843906110BD526A82
:10156000446D1A402280426D921C42654A8B521E85
:101570004A83498B0029F1D101680A68FF2321338E
:101580009A430A6001688A68520852008A602021E2
:10159000816700210166FFF73DFD10BD10B50146D2
:1015A00040318B8B846F0268222C04D09069082113
:1015B0000843906110BD526A1A40436D1A70426D23
:1015C000521C42654A8B521E4A83498B0029F1D135
:1015D00001680A68FF2321339A430A6001688A6818
:1015E000520852008A602021816700210166FFF7BE
:1015F00011FD10BDF8B504462669A268E7693243BB
:101600006669102000253E432368324378491E68EE
:10161000784F3E4016431E6023685A6803263603FF
:10162000B243E66832435A602368A2698B4201D014
:10163000266A32439E680B273F02BE4316439E60D4
:101640006D4E23686D4AB3420CD1D2689207920F57
:1016500006D0012A38D0022A34D0032A20D11EE035
:1016600001201DE0664EB3420AD1D2680C263240FA
:1016700026D0042A28D0082A24D00C2A10D10EE023
:101680008B420DD1D66803229202164018D0012257
:101690009202B61A18D0B61A14D0964200D1082079
:1016A000564A0126403A574FF6038B4236D100285E
:1016B0000CD002280DD0042812D008281FD11CE01D
:1016C0000020EDE70220EBE70420E9E7FFF74CF804
:1016D00008E01068C00601D5384605E04A4803E036
:1016E000FFF762F8002873D06268510051188142F8
:1016F00005D81103814202D303E03046F4E7012507
:1017000066E0010E06025008002330185941FEF72A
:1017100007FD03210902411A3C4A55E0E169B14243
:1017200032D1030000F00AF909070A0D0625060662
:10173000062B0600E3E7FFF717F81CE0FFF724F895
:1017400019E010686168C00602D54808304A01E017
:10175000304A48088018FEF7CDFC80B201462E4A78
:1017600010399142CBD8511C01400007400F08436B
:101770002CE0FFF719F8616840004A08EAE7616861
:10178000012248081204E5E7030000F0D7F8090732
:101790000A0D06260606062C0600B0E7FEF7E4FF53
:1017A0001DE0FEF7F1FF1AE010686168C00602D57F
:1017B0004808C01902E014484A081018FEF79AFCBD
:1017C00080B20146144A1039914298D82168C86005
:1017D0000020206660662846F8BDFEF7E5FF6168D8
:1017E0004A088018EAE7616848088019E6E70000BF
:1017F00000480040F369FFEF00380140401002400C
:101800000044004000093D000024F400FFFC0F00EC
:1018100000127A000048E801EFFF0000416F212923
:1018200010D1014640314A8A002A0CD0C26C0368AC
:101830001288D205D20D9A62C26C921CC264488A88
:10184000401E4882704701680A6880239A430A60F4
:10185000006801684022114301607047416F2129EF
:101860000ED1014640314A8A002A0AD0C26C036870
:1018700012789A62C26C521CC264488A401E488226
:10188000704701680A6880239A430A60006801680B
:101890004022114301607047FFB581B017460E46E4
:1018A00004460A9D09E0681C07D0FEF7A1FD0499D3
:1018B000401AA8420CD8002D0AD02068C1693046D1
:1018C000884318D00020B842EDD0002005B0F0BD0C
:1018D00020680168FF22A13291430160206881687D
:1018E00049084900816020206067A06700206034BB
:1018F00020740320EAE70120E5E7000010B5024864
:10190000FFF7FCF910BD00005800002010B5024898
:10191000FFF7F4F910BD0000D80000200FB410B597
:1019200003A9044B044A029800F024F810BC08BC38
:1019300004B01847C51A00081800002030B47446D7
:10194000641E2578641CAB4200D21D46635D5B00BB
:10195000E31830BC184702E008C8121F08C1002A6B
:10196000FAD170477047002001E001C1121F002A20
:10197000FBD17047FFB58DB00446002506E0252851
:101980000AD0109A0F999047641C6D1C207800288B
:10199000F5D1284611B0F0BD00270121484A009733
:1019A00000E00743641C23780846203B984010421F
:1019B000F7D120782E2817D1042007436078641CC3
:1019C0002A280CD10E98641C02C800910E900BE0DE
:1019D00000990A22514330394018641C0090207845
:1019E000014630390929F3D920780028D1D064285C
:1019F00008D0692806D075281ED0109A0F999047F4
:101A00006D1C5BE00A200E99019001C90E9100281F
:101A100002DA40422D2102E0390504D52B216A4625
:101A20001172012103E0F90704D02021F7E70BAE82
:101A30000B910DE00021FAE70A200E99019001C9EF
:101A40000E91F7E70199FEF755FB3031761E3170A4
:101A50000028F7D103A8801B20300190780701D51A
:101A6000009801E0012000900199884201DD401AB0
:101A700000E000200027009006E002A8109AC05D58
:101A80000F9990476D1C7F1C0B988742F5DB04E093
:101A9000109A30200F9990476D1C0099481E0090B5
:101AA0000029F5DC05E03078109A761C0F999047F4
:101AB0006D1C0199481E01900029F4DC641C65E747
:101AC0000928010001B5044B012269460348FFF7CC
:101AD000C5FA009808BD0000FFFF00005800002074
:101AE000FEF794FCFFF7F0FBFFF75EFBFFF78AFBC6
:101AF000FFF766FBFFF7A2FB074C062207490848E1
:101B0000FFF714FB05490822891D0548FFF720FA55
:101B10002046FEF7A2FBF0E710270000020000209D
:101B2000D8000020000000000000000001020304B3
:101B300006070809030406080C10182030000000EE
:101B40000001020304000000681B000800000020E0
:101B50001C00000056190008841B00081C0000200F
:101B60003C05000066190008000055AA1100021289
:101B70000000000000000000000000000000200045
:041B80000000000061
:04000005080000C12E
:00000001FF
